:040000000CEF00F011
:10000800FACF01F1FBCF02F1E9CF03F11BED00F0CC
:1000180000EE00F010EE01F014EC00F068EF00F0D4
:10002800EE6AE550E150FCE1E250FAE11200060008
:10003800EACF04F1E1CF05F1E2CF06F1D9CF07F11C
:10004800DACF08F1F3CF09F1F4CF0AF1F6CF0BF1CB
:10005800F7CF0CF1F8CF0DF1F2AA01D001D019D0E9
:10006800F2A401D001D015D0002A00504C0AD8A41F
:1000780001D001D00DD081B201D001D002D081824F
:1000880001D081920101006F000E006E0101005144
:10009800F2940DC1F8FF0CC1F7FF0BC1F6FF0AC1BE
:1000A800F4FF09C1F3FF08C1DAFF07C1D9FF06C190
:1000B800E2FF05C1E1FF04C1EAFF03C1E9FF02C194
:1000C800FBFF01C1FAFF1100D580D582D584D596F2
:1000D800D59AD58CF28AF28CF28ED58E9392FFD770
:0400E8000CEF00F029
:020000040030CA
:0A00000000021F1E0081C1000FC0A6
:00000001FF
